:100000000C947B020C94BF020C94BF020C94BF02B0
:100010000C94BF020C94BF020C94BF020C94BF025C
:100020000C94BF020C94BF020C94E90D0C94BB0E0F
:100030000C94BF020C94BF020C94BF020C94BF023C
:100040000C94BF020C9475210C94BF020C94BF0257
:100050000C94BF020C94571C0C94BF020C94BF026A
:100060000C94BF020C94BF020C94BF020C94BF020C
:100070000C94BF020C94BF020C94BF020C94BF02FC
:100080000C94BF020C94BF020C94BF020C94BF02EC
:100090000C94BF020C94BF020C94BF020C94BF02DC
:1000A0000C94BF020C94BF020C94BF02280F4A0F9D
:1000B00038104A0F38108F0FB20F381007101A106F
:1000C000E912E912181318134E136E139F149F149C
:1000D00079139F142914291490149F149F149914B0
:1000E00036143614361436143614361436143614C0
:1000F00036143614361436143614361436143614B0
:10010000481455145C1463146D140000F0A12E0003
:100110004C002A00E100354100001E000E000B00DB
:100120001B6134004D001F00370004001400E1047F
:100130002800200012000800340050002C0021008C
:1001400036000C002F004F004A0022001D0018004E
:10015000330000006564500001530000006F000090
:10016000E3004F000153000000670000E20023009D
:100170001900070005000000296124000A0017008B
:10018000130052004B002500060015001A00510014
:10019000E50026000F00110010002F002B002700A3
:1001A0002D0016420D6130004E002D001C00096824
:1001B000E500C10000000100010001000100010094
:1001C00000003A001E0220022202010001003B0052
:1001D0001F0221022302010001003C002F0226021F
:1001E0002F00010001003D00300227023000010015
:1001F00001003E003102350035020000010001001F
:1002000001000000010000000100010001000000E9
:100210000100000001003F005200510024020000D4
:1002200001004000240021001E00010001004100E7
:10023000250022001F003700010042002600230095
:10024000200027000100430025022E0231002E006D
:100250000100440045000100010001000000010010
:100260000100010001000100000001000100010087
:1002700001000100010001000100F2000100010085
:1002800001000100F000F1000100F4000100010094
:100290000100F3000100F500010001000100010070
:1002A0000100000001000100010000000100000049
:1002B0000100010001000000010000000100010038
:1002C0000100010001000000010001000100010027
:1002D0000100A9000100010001000100AC00AA001A
:1002E000B600010001000100AB00A8000100010000
:1002F0000100010001000100010001000100AE0049
:1003000001000100000016034500720067006F0045
:1003100044006F007800200045005A0000001603DA
:100320004500720067006F0044006F0078002000F5
:1003300045005A0000000403090409026D0004018D
:1003400000A0FA09040000010301010009211101C4
:1003500000012240000705810308000A090401008A
:100360000103010200092111010001224D000705CE
:10037000820308000A0904020001030000000921A9
:10038000110100012236000705830308000A090451
:1003900003000103000000092111010001223900BE
:1003A000070584031000011201100100000008ED90
:1003B000FE071301000102000105010906A1010564
:1003C0000719E029E7150025019508750181020547
:1003D000081901290595057501910295017503918B
:1003E0000105071900297715002501957875018108
:1003F00002C005010980A101850216010026B7008F
:100400001A01002AB700751095018100C0050C097A
:1004100001A1018503160100269C021A01002A9CF5
:1004200002751095018100C005010902A1010901B1
:10043000A10005091901290515002501950575017A
:10044000810295017503810105010930093115818A
:10045000257F95027508810609381581257F95014C
:1004600075088106050C0A38021581257F950175EE
:10047000088106C0C005010906A101050719E02988
:10048000E715002501950875018102950175088120
:100490000105081901290595057501910295017558
:1004A0000391010507190029FF150026FF00950695
:1004B00075088100C000000000000000000000007E
:1004C000010204060A0F17202C3A4A5D71879DB37A
:1004D000C7DAE9F5FCFFFCF5E9DAC7B39D87715D82
:1004E0004A3A2C20170F0A060402010000000000FF
:1004F00000000000000011241FBECFEFDAE0DEBFD5
:10050000CDBF04B603FE24C08091FD019091FE0191
:10051000A091FF01B09100028730904BA740B04BF3
:10052000B9F41092FD011092FE011092FF01109299
:10053000000214BE84B7877F84BF88E10FB6F894A9
:1005400080936000109260000FBEE0E0FFE3099529
:1005500011E0A0E0B1E0E8E7F6E402C005900D92FA
:10056000A433B107D9F711E0A4E3B1E001C01D92B3
:10057000AD3FB107E1F70E94310B0C943A230C9484
:1005800000001092B9008AE08093B800089594EAC0
:100590009093BC009091BC0097FFFCCF9091B90064
:1005A000987F983021F0903111F081E00895809388
:1005B000BB0084E88093BC008091BC0087FFFCCF27
:1005C0008091B900887F883111F0803471F780E024
:1005D000089584E98093BC008091BC0084FDFCCF29
:1005E00008958093BB0084E88093BC008091BC0098
:1005F00087FFFCCF9091B900987F81E0983209F491
:1006000080E0089584E88093BC008091BC0087FF5F
:10061000FCCF8091BB00089580B38C7080BB81B308
:10062000836F81BB089580910101811115C080E421
:100630000E94C7028093010181110CC082E10E94D7
:10064000F10280930101811105C08FEF0E94F10238
:10065000809301010E94E90284B1807F84B985B151
:10066000807F85B98AB1837F8AB98BB1837F8BB94B
:100670003E98469808950E94DD04809301010E94EF
:1006800013030E940C03A5E3B1E0E3E4F1E08EE084
:100690008E0F11921D928E13FCCF0C94C7040E94F2
:1006A000DD04809301010E9413030E940C03A5E363
:1006B000B1E0E3E4F1E08EE08E0F11921D928E1313
:1006C000FCCF0895BF92CF92DF92EF92FF920F93EB
:1006D0001F93CF93DF9380910101882379F080915C
:1006E00034018F5F80933401811108C00E94DD04C2
:1006F00080930101811102C00E946F0405E311E0A3
:10070000C0E0D0E0DD24D39482E0C82EEE24E39450
:10071000F12CC730D10500F580910101811164C031
:1007200080E40E94C70280930101811112C082E11E
:100730000E94F1028093010181110BC0C7010C2EB0
:1007400001C0880F0A94EAF780950E94F102809315
:1007500001010E94E90248C0CA30A1F028F4C83063
:1007600059F0C93061F005C0CC3089F070F0CD305F
:1007700089F0209A289810C0219A29980DC0229AB1
:100780002A980AC0239A2B9807C0529A01C0539AFC
:100790005B9802C03E9A469890EA9A95F1F79FB10D
:1007A000799902C082E001C080E091709D25982B6C
:1007B0007C9902C084E001C080E0892B7D9902C051
:1007C00038E001C030E0832B7E9902C020E101C0F7
:1007D00020E0822B9FB19095991F9927991F9295A0
:1007E000990F907E892B0FC080910101811149C022
:1007F00080E40E94C70280930101882379F1B12C23
:100800000E94E9028B2DF8019081981719F08083DE
:10081000C09200010E94130321960F5F1F4FCE303C
:10082000D10509F076CF80910001882361F18150D4
:1008300080930001882339F08FE99FE00197F1F759
:1008400000C0000020C0A3E4B1E0E5E3F1E0CF0187
:10085000825F91919D938E13FCCF15C083E10E941E
:10086000F102809301018111CACF81E40E94C70285
:10087000809301018111C3CF0E940203B82EB0946E
:10088000BFCF80E0C0CF0E946D0481E0DF91CF91A7
:100890001F910F91FF90EF90DF90CF90BF90089540
:1008A000E82FF0E0ED5BFE4F8081089508950F93EF
:1008B0001F93CF93DF93C3E4D1E010E00C2F025FCE
:1008C000899190E00E947E1B180F0C13F9CF812FA5
:1008D000DF91CF911F910F9108950C943D0556988B
:1008E0005E9825982D9826982E9827982F988FEF08
:1008F00090E0909389008093880090938B00809380
:100900008A0090938D0080938C00259A2D9A2FEF6A
:1009100080E792E0215080409040E1F700C0000065
:10092000269A2E9A2FEF80E792E021508040904047
:10093000E1F700C00000279A2F9A2FEF80E792E09E
:10094000215080409040E1F700C0000025982D988C
:100950002FEF80E792E0215080409040E1F700C007
:10096000000026982E982FEF80E792E021508040DB
:100970009040E1F700C0000027982F9856985E98A5
:1009800025982D9826982E9827982F98089589EACB
:100990008093800089E08093810024982C983F9870
:1009A0008AB18F748AB96E98479A8BB1806B8BB974
:1009B000769A0E946F040C943C0580E280930101BA
:1009C0008091510181110EC00E94C10281E080938B
:1009D00051012FEF83ED90E3215080409040E1F7EB
:1009E00000C0000080E40E94C702809301018111D1
:1009F0002EC00E94F10280930101811128C00E9443
:100A0000F10280930101811122C08FE30E94F10263
:100A10008093010181111BC00E94E90280E40E94C1
:100A2000C70280930101811112C08CE00E94F10283
:100A30008093010181110BC00E94F102809301019A
:100A4000811105C08FE30E94F102809301010E9491
:100A5000E90280910101089561110BC0FC018281BE
:100A6000882321F085EE0E948D1103C085EE0E943F
:100A7000551280E090E0089508956091BE01709154
:100A8000BF018091C0019091C1010E948A1B5698BC
:100A90005E9825982D9826982E9827982F98813023
:100AA00019F0823021F00895259A2D9A0895269AFA
:100AB0002E9A089581E0089581E008950C945C05D4
:100AC0000895282F882339F090E02A3010F44D96AD
:100AD00008950697089587E290E00895AF92BF9237
:100AE000DF92EF92FF920F931F93CF93DF938C01CE
:100AF000FC01C081D181CE010E94031ABE010E9477
:100B0000DE08EC01B8010E945E05882309F4C9C122
:100B1000F8018281882309F4BEC080915E018111B1
:100B20001FC0C431F0E7DF0709F0B5C10E946005BE
:100B300081E080935E010E94211C90935D0180936F
:100B40005C011092550110925701109256011092BB
:100B500059011092580110925B0110925A01A1C1E3
:100B600080915C0190915D010E942D1C883C910553
:100B700070F480915501E82FF0E0EE0FFF1FEA5A64
:100B8000FE4FD183C0838F5F809355018AC1C130EE
:100B900020E8D20708F451C0F8018281882309F4C3
:100BA0007EC05E01E894B7F880915401813079F0FD
:100BB00050F08230C1F482EE0E948D1187E50E94D0
:100BC0008D1187E50EC082EE0E948D110CC080EE63
:100BD0000E948D1181EE0E948D1188E10E948D117D
:100BE00088E10E9455128CE0E82EF12CC5010E2CF4
:100BF00002C0969587950A94E2F78F700E9461056E
:100C0000D82E0E948D118D2D0E945512F4E0EF1AFE
:100C1000F1082CEFE2162FEFF20641F78091540114
:100C2000813029F010F0823041F482EE04C080EE71
:100C30000E94551281EE0E945512C43180E7D807F8
:100C400068F4C23090E7D90708F046C0C115E0E764
:100C5000DE0771F0C130D047A1F10CC1C33320E7EA
:100C6000D20709F4D8C0C433D04709F4EBC002C19D
:100C7000F8018281882309F402C10E940A15FFEF5E
:100C800024E38CE0F15020408040E1F700C00000F8
:100C90000E947C1C06C1C13080E8D80770F2C431C4
:100CA00020E7D20708F0B3C0C23080E7D807A0F42D
:100CB000C11590E7D90709F4E2C0C130D04709F067
:100CC000D9C0F8018281882309F4D9C08091DB0161
:100CD00081608093DB01E5C0F8018281882309F4FB
:100CE000CEC00E94D61C811102C00E94BC1C0E9472
:100CF000E91C90E09093EF018093EE01C230F0E7A1
:100D0000DF0721F48091EE0181607AC0C33020E7D3
:100D1000D20721F48091EE01826072C0C43080E776
:100D2000D80721F48091EE0184606AC0C53090E755
:100D3000D90719F48091EE0127C0C630E0E7DE073D
:100D400021F48091EE0180615BC0C730F0E7DF07DE
:100D500021F48091EE01806253C0C83020E7D207B1
:100D600021F48091EE0180644BC0C93080E7D80740
:100D700021F48091EE01806843C0CA3090E7D90722
:100D800029F48091EE01846088603AC0CB30E0E7BE
:100D9000DE0721F48091EE018E7F32C0CC30F0E787
:100DA000DF0721F48091EE018D7F2AC0CD3020E74E
:100DB000D20721F48091EE018B7F22C0CE3080E7F4
:100DC000D80719F48091EE011AC08091EE01CF305E
:100DD00090E7D90711F48F7E13C0C031E0E7DE073A
:100DE00011F48F7D0DC0C131F0E7DF0711F48F7B67
:100DF00007C0C231D04711F48F7702C08B7F877F45
:100E00008093EE018091EE010E94ED1C4AC0C33335
:100E1000F0E7DF07A1F4F8018281882321F0109226
:100E2000520182E016C080915201811106C086E213
:100E30000E948D1186E20E94551282E018C0C433D0
:100E4000D047C1F4F8018281882331F01092530118
:100E500080E20E94A41225C080915301811106C036
:100E600087E20E948D1187E20E94551280E20E9463
:100E7000AB1217C081E08093520180935301C801E7
:100E8000DF91CF911F910F91FF90EF90DF90BF9076
:100E9000AF900C945A05C130F0E8DF0708F081CE1E
:100EA000CCCE80E0DF91CF911F910F91FF90EF901A
:100EB000DF90BF90AF90089526E0729FF00111245B
:100EC00044E5849FE00DF11D1124E60FF11DEE0FA6
:100ED000FF1FE25FFE4F859194910E94F0088115FB
:100EE00060E49607B0F5811570E3970708F0DEC05F
:100EF000803E9105D8F4803C910508F06CC0883A9A
:100F0000910578F4853A910508F06BC08130910520
:100F100009F452C108F40FC18430910508F04CC1A6
:100F20000AC18B3B910508F467C005C18F3F91054D
:100F300009F048F4803F910508F0ADC0883E910566
:100F400008F43AC1F8C0811520E2920708F0A5C064
:100F50000895811543E5940790F4811562E596079D
:100F600008F0C8C0811571E5970708F0BEC081156B
:100F700020E5920708F09DC09F70906A0895811542
:100F800045E59407D8F4811564E5960708F0C8C0D4
:100F9000482F4695469570E2479FA0011124837023
:100FA000992721E030E0B90102C0660F771F8A95CA
:100FB000E2F7CB01842B952B9A680895811576E58D
:100FC000970708F4B2C09C0130562115304108F053
:100FD000B2C09F70AEC0FC01EE0FFF1FE657F0409D
:100FE00062C0853A910509F4A9C0863A910509F0D5
:100FF000A8C082E890E40895883A910509F4A4C055
:10100000893A910509F4A3C08A3A910509F4A2C06E
:101010008B3A910509F4A1C08C3A910509F4A0C05E
:101020008D3A910509F49FC0803B910509F49EC05B
:101030008E3A910509F49DC08F3A910509F49CC040
:10104000813B910509F49BC0823B910509F49AC04C
:10105000833B910509F499C0843B910509F498C03C
:10106000853B910509F497C0863B910509F496C02C
:10107000873B910509F495C0883B910509F494C01C
:10108000893B910509F493C08A3B910509F492C00C
:1010900080E094E4089590650895FC01FF70EE0FE0
:1010A000FF1FE65FFE4F8591949108959927906CFC
:1010B0000895482F437021E030E002C0220F331F13
:1010C0004A95E2F73C68AC0164E0569547956A950D
:1010D000E1F74370342B8F708695869560E2869F8A
:1010E000C0011124822B932B0895982F8827816F9C
:1010F000906A0895482F4695469570E2479FA00153
:1011000011248370992721E030E0B90102C0660FF5
:10111000771F8A95E2F7CB01842B952B9C68089565
:10112000982F8827846F906A08958F719927982F38
:1011300088279062089580E090E0089581E890E427
:10114000089583E890E4089582EE94E4089589EE8A
:1011500094E408958AEE94E4089585EB94E4089568
:1011600086EB94E4089587EB94E408958CEC94E482
:1011700008958DEC94E4089583E895E408958AE851
:1011800095E4089582E995E4089584E995E4089545
:1011900081E296E4089583E296E4089584E296E479
:1011A000089585E296E4089586E296E4089587E23C
:1011B00096E408958AE296E40895089596E0799F6A
:1011C000F001112494E5899FE00DF11D1124E60F33
:1011D000F11DEE0FFF1FE25FFE4F85919491089580
:1011E0008238910549F1B0F48133910509F458C072
:1011F00048F48932910509F44EC08A32910509F408
:1012000054C008958533910509F440C08933910590
:1012100099F00895833E910529F138F4803E9105B7
:1012200091F0823E9105A1F00895863E9105F9F076
:10123000873E910531F108952091EE0120FD3AC0DD
:1012400021FD38C008958091EE0180FD35C032C087
:101250008091EE0182FF32C08091EE0184FD30C0AA
:1012600083EE39C08091EE0182FD28C0F5CF8091D8
:10127000EE0183FF27C08091EE0184FD21C087EE3F
:101280002AC08091EE0183FD1DC0F5CF8091EE0153
:1012900085FD1AC01BC08091EE0185FD17C014C0EA
:1012A0008091EE0186FD14C015C08091EE0186FD8F
:1012B00011C00EC080EE0FC089E30DC082EE0BC0DE
:1012C00080E009C086EE07C089E205C085E303C05F
:1012D0008AE201C081E390E0089508950C946D09BD
:1012E00080916F010895CF93DF9300D01F92CDB707
:1012F000DEB79C018091F401843019F593E0998365
:101300003B832A839093E9008FEF9091E80081500E
:1013100095FD06C095ED9A95F1F700008111F5CF86
:101320008091E80085FF0DC040E050E063E070E090
:10133000CE0101960E94D90B8091E8008E778093B0
:10134000E8000F900F900F90DF91CF910895CF9309
:10135000DF9300D01F92CDB7DEB72091F401243087
:1013600021F522E029839B838A8383E08093E9002F
:101370008FEF9091E800815095FD06C095ED9A950C
:10138000F1F700008111F5CF8091E80085FF0DC0D5
:1013900040E050E063E070E0CE0101960E94D90B7E
:1013A0008091E8008E778093E8000F900F900F9067
:1013B000DF91CF9108952091F4012430F1F422E0DF
:1013C0002093E9002FEF3091E800215035FD06C051
:1013D00035ED3A95F1F700002111F5CF2091E800A5
:1013E00025FF0BC040E050E065E070E00E94D90BA3
:1013F0008091E8008E778093E8000895CF93DF9383
:10140000EC019091F401943009F046C080910C01F8
:101410008823D9F080910D018823B9F09093E900D9
:101420008FEF9091E800815095FD06C095E19A9567
:10143000F1F700008111F5CF8091E80085FF2CC005
:1014400040E050E060E170E017C081E08093E90087
:101450008FEF9091E800815095FD06C095ED9A952B
:10146000F1F700008111F5CF8091E80085FF14C0ED
:1014700040E050E068E070E0CE010E94D90B80911E
:10148000E8008E778093E80080E1FE01AFE5B1E0EF
:1014900001900D928A95E1F7DF91CF9108958091A7
:1014A000F301811109C00E946E0D0E94CB0D809145
:1014B000E20084608093E20008951092F3010895A1
:1014C00008950C9462210E94121C0E9468210E94BF
:1014D00071100C946E0942E061EC81E00E94E80C0E
:1014E00042E061EC82E00E94E80C42E061EC83E0C3
:1014F0000E94E80C42E161EC84E00C94E80C8091DD
:10150000F601833009F455C030F4813071F0823037
:1015100009F48EC008958A3009F47AC08B3009F43A
:1015200060C0893009F09CC020C08091F501813AEB
:1015300009F096C08091E800877F8093E800809151
:10154000F9019091FA01892B21F460E18FE591E096
:1015500003C060E080E090E070E00E94240C809185
:10156000E8008B778093E80008958091F50181323F
:1015700009F076C08091F9019091FA01009719F075
:10158000039709F06DC08091E800877F8093E800A1
:101590008091E80082FD05C08091F4018111F8CFAF
:1015A0005FC08091F10080936F018091E8008B779C
:1015B00053C08091F501813A09F052C08091F90140
:1015C0009091FA01892B09F04BC08091E800877F48
:1015D0008093E8008091E80080FFFCCF80910C01AF
:1015E00036C08091F5018132D9F58091F901909151
:1015F000FA01892BA9F58091E800877F8093E800A4
:101600000E941D0D8091F70180930C010C940A1526
:101610008091F501813221F58091E800877F8093E8
:10162000E8000E941D0D8091F801809370010895DB
:101630008091F501813AA1F48091E800877F809341
:10164000E8008091E80080FFFCCF809170018093DA
:10165000F1008091E8008E778093E8000C941D0DD6
:10166000089584B7877F84BF88E10FB6F89480938C
:101670006000109260000FBE80E8809361001092BD
:1016800061000E94C0100E946E0D0E94CB0D8091DF
:10169000E20084608093E20078940E9451100E94DE
:1016A000C21082E091E00E946C100E945021809153
:1016B000F401853069F40E94DA1B8091F2018823DD
:1016C000B1F30E94041C882391F30E94C30BEFCF57
:1016D0000E94C810ECCF292F332723303105C9F0E1
:1016E00064F42130310581F02230310509F043C026
:1016F0008DE690E02AE333E042C021323105F1F07B
:101700002232310541F137C082E190E027EA33E02F
:1017100036C099278130910541F08230910541F022
:10172000892B49F5E6E3F3E005C0EEE1F3E002C002
:10173000E6E0F3E0849190E09F0121C06430D8F4AA
:10174000E62FF0E0EE0FFF1FEE5DFE4F20813181AE
:1017500089E090E014C0643070F470E0FB01EE0F9B
:10176000FF1FE65EFE4F20813181FB01EA5EFE4FE6
:10177000808190E004C080E090E020E030E0FA0159
:1017800031832083089580E189BD82E189BD09B458
:1017900000FEFDCF8091D8008F7D8093D80080918E
:1017A000E00082608093E0008091E00081FDFCCF4A
:1017B0000895CF92DF92EF92FF920F931F93CF93F2
:1017C000DF93EC018B016A010E943C0D811133C053
:1017D000C114D10439F0F60180819181081B190BE5
:1017E000C80FD91FE12CF12C0115110519F18091B9
:1017F000E80085FD16C08091E8008E778093E800B0
:10180000C114D10449F0F60180819181E80EF91EDE
:10181000F182E08285E00FC00E943C0D882321F315
:101820000AC089918093F10001501109FFEFEF1A6E
:10183000FF0ADACF80E0DF91CF911F910F91FF90E7
:10184000EF90DF90CF9008952091FB013091FC0143
:101850002617370748F06115710539F42091E80023
:101860002E772093E80001C0B90140E061157105B1
:10187000A9F12091F401222309F443C0253009F491
:1018800042C02091E80023FD40C02091E80022FDE5
:1018900032C02091E80020FFE9CF4091F300209171
:1018A000F20030E0342BFC01CF016115710559F0D5
:1018B0002830310540F481918093F1006150710925
:1018C0002F5F3F4FF1CF41E02830310509F040E074
:1018D0002091E8002E772093E800C8CF4111C9CFAE
:1018E0000AC08091F401882361F0853061F0809115
:1018F000E80083FD0AC08091E80082FFF2CF80E01B
:10190000089582E0089583E0089581E0089520918C
:10191000FB013091FC012617370748F0611571056E
:1019200039F42091E8002E772093E80001C0B90136
:10193000FC0120E06115710591F18091F40188238B
:1019400009F440C0853009F43FC08091E80083FD70
:101950003DC08091E80082FD2FC08091E80080FFAB
:10196000E9CF2091F3008091F20090E0922B611575
:10197000710559F08830910540F424912093F100CD
:101980003196615071090196F2CF21E0089709F074
:1019900020E08091E8008E778093E800CBCF211182
:1019A000CCCF0AC08091F401882361F0853061F0CA
:1019B0008091E80083FD0AC08091E80082FFF2CFA9
:1019C00080E0089582E0089583E0089581E008951D
:1019D000982F973058F59093E900981739F0709147
:1019E000EC002091ED005091F00003C0242F762FE1
:1019F00050E021FF19C03091EB003E7F3093EB00A7
:101A00003091ED003D7F3093ED003091EB0031607F
:101A10003093EB007093EC002093ED005093F000B6
:101A20002091EE0027FF07C09F5FD3CF8F70809378
:101A3000E90081E0089580E008958091F50187FF35
:101A400011C08091E80082FD05C08091F4018111F0
:101A5000F8CF11C08091E8008B770BC08091F40122
:101A6000882349F08091E80080FFF8CF8091E8005A
:101A70008E778093E80008952091E4003091E5008E
:101A800095E64091EC00842F817040FF22C0809148
:101A9000E80080FD1CC08091F401882391F085301E
:101AA00091F08091EB0085FD10C04091E4005091D1
:101AB000E5004217530729F39A01915011F784E08A
:101AC000089582E0089583E0089581E0089580E01C
:101AD00008954091E80042FFDECF08950E94DC0D9A
:101AE0000E94E40DE0EEF0E0808181608083E8ED0B
:101AF000F0E080818F77808319BCA7EDB0E08C91F6
:101B00008E7F8C9380818F7E80831092F301089565
:101B10000F931F93CF93DF930E94DC0D0E94E40D7F
:101B2000C8EDD0E088818F7788838881806888833A
:101B300088818F7D888319BC1092F4011092F00186
:101B40001092F2011092F10100EE10E0F801808194
:101B50008B7F808388818160888342E060E080E0C1
:101B60000E94E80CE1EEF0E080818E7F8083E2EE5F
:101B7000F0E0808181608083808188608083F801CB
:101B800080818E7F8083888180618883DF91CF917F
:101B90001F910F910895E8EDF0E080818F7E8083A2
:101BA000E7EDF0E080818160808384E082BF81E0A6
:101BB0008093F3010C94880DE8EDF0E080818E7F36
:101BC00080831092E20008951092DA001092E100F2
:101BD00008951F920F920FB60F9211242F933F93E7
:101BE0004F935F936F937F938F939F93AF93BF9325
:101BF000EF93FF938091E10082FF0BC08091E200A0
:101C000082FF07C08091E1008B7F8093E1000E94FA
:101C100050108091DA0080FF1FC08091D80080FFB3
:101C20001BC08091DA008E7F8093DA008091D9000A
:101C300080FF0DC080E189BD82E189BD09B400FE4D
:101C4000FDCF81E08093F4010E944F0A05C019BCCA
:101C50001092F4010E945D0A8091E10080FF19C09A
:101C60008091E20080FF15C08091E2008E7F80931A
:101C7000E2008091E20080618093E2008091D800D0
:101C800080628093D80019BC85E08093F4010E94A3
:101C9000610A8091E10084FF30C08091E20084FFFE
:101CA0002CC080E189BD82E189BD09B400FEFDCF71
:101CB0008091D8008F7D8093D8008091E1008F7E45
:101CC0008093E1008091E2008F7E8093E20080911A
:101CD000E20081608093E2008091F001882311F09E
:101CE00084E007C08091E30087FD02C081E001C06D
:101CF00083E08093F4010E94630A8091E10083FFF6
:101D000029C08091E20083FF25C08091E100877F98
:101D10008093E10082E08093F4011092F0018091C1
:101D2000E1008E7F8093E1008091E2008E7F8093BE
:101D3000E2008091E20080618093E20042E060E096
:101D400080E00E94E80C8091F00088608093F000B1
:101D50000E94600AFF91EF91BF91AF919F918F9187
:101D60007F916F915F914F913F912F910F900FBE97
:101D70000F901F9018951F920F920FB60F9211247B
:101D80002F933F934F935F936F937F938F939F9383
:101D9000AF93BF93CF93DF93EF93FF93C091E9008D
:101DA000CF708091EC00D82FD17080FDD0E81092D8
:101DB000E9008091F000877F8093F00078940E9482
:101DC000FF0E1092E9008091F00088608093F0008F
:101DD000CD2BCF70C093E900FF91EF91DF91CF91B0
:101DE000BF91AF919F918F917F916F915F914F9133
:101DF0003F912F910F900FBE0F901F9018951F933A
:101E0000CF93DF93CDB7DEB7AA970FB6F894DEBFB6
:101E10000FBECDBFE5EFF1E088E08E0F9091F100AD
:101E200091938E13FBCF0E947F0A8091E80083FF7D
:101E30001FC18091F5019091F601492F50E04A3081
:101E4000510508F015C1FA01EA5AFF4F0C94EA2235
:101E5000803881F0823809F00BC18091F9018F70D0
:101E60008093E9008091EB0085FB882780F9109230
:101E7000E90006C08091F1019091F2019111826018
:101E80009091E800977F9093E8008093F100109282
:101E9000F100C8C0282F2D7F09F0EAC0882319F06F
:101EA000823061F0E5C08091F701813009F0E0C037
:101EB000933009F080E08093F2012BC08091F7010C
:101EC000811127C08091F9018F7009F4D1C08093EE
:101ED000E9002091EB0020FF1CC0933021F4809199
:101EE000EB00806214C09091EB0090619093EB0046
:101EF00021E030E0A90102C0440F551F8A95E2F7A6
:101F00004093EA001092EA008091EB008860809391
:101F1000EB001092E9008091E800877F86C0811174
:101F2000A7C01091F7011F778091E3008078812B83
:101F30008093E3008091E800877F8093E8000E940F
:101F40001D0D8091E80080FFFCCF8091E300806848
:101F50008093E300111102C082E001C083E080930E
:101F6000F40186C08058823008F082C08091F70169
:101F70009091F8018C3D53E0950779F583E08A83D1
:101F80008AE289834FB7F894DE01139620E03EE0A1
:101F900051E2E32FF0E050935700E49120FF03C09B
:101FA000E295EF703F5FEF708E2F90E0EA3010F017
:101FB000C79601C0C0968D939D932F5F243149F73A
:101FC0004FBF8091E800877F8093E8006AE270E06D
:101FD000CE0101960E94240C14C0AE014F5F5F4FEA
:101FE0006091F9010E946B0BBC01009709F440C09D
:101FF0009091E800977F9093E80089819A810E94F0
:10200000870C8091E8008B778093E80031C080389E
:1020100079F58091E800877F8093E8008091F00156
:102020008093F1008091E8008E778093E8000E9411
:102030001D0D1EC081111CC09091F7019230C0F49B
:102040008091E800877F8093E8009093F0010E94E0
:102050001D0D8091F001811106C08091E30087FD84
:1020600002C081E001C084E08093F4010E946B0A09
:102070008091E80083FF0AC08091E800877F809309
:10208000E8008091EB0080628093EB00AA960FB687
:10209000F894DEBF0FBECDBFDF91CF911F910895A1
:1020A0000895CF938091F4018823A1F0C091E900B5
:1020B000CF709091EC00892F817090FD80E8C82B43
:1020C0001092E9008091E80083FD0E94FF0ECF701E
:1020D000C093E900CF9108959093760180937501A4
:1020E0000895E0917501F0917601309721F001900B
:1020F000F081E02D099480E00895E0917501F09160
:102100007601309721F00280F381E02D0994089543
:10211000E0917501F0917601309721F00480F5810E
:10212000E02D099408952091730130917401821774
:10213000930771F09093740180937301E09175019E
:10214000F0917601309721F00680F781E02D099417
:10215000089520917101309172018217930771F0F7
:102160009093720180937101E0917501F091760175
:10217000309721F00084F185E02D099408950895A9
:102180000C94BF100E94181C0E943B030C949E1CD0
:102190009F92AF92BF92CF92DF92EF92FF920F93F6
:1021A0001F93CF93DF9300D000D000D0CDB7DEB720
:1021B0000E9462030DE010E0AA24A394B12C902E9B
:1021C000802F0E945004980128583E4F6901F90160
:1021D000F080F826A1F40150110988F78FEF898368
:1021E0008A831B820E94211C8160782F9D838C83AF
:1021F00049815A816B818D810E945F112FC090911E
:10220000DB0191FF04C08E830E9456048E8125E07D
:1022100030E0A501022E01C0440F0A94EAF7E42E33
:102220004F21C1F029839A828E2191E009F490E038
:102230009B830E94211C8160782F9D838C83498120
:102240005A816B818D810E945F11F6018081E826A1
:10225000E08204C021503109E0F6BDCF0E946C1E1F
:10226000109177010E9471101817B9F00E94711037
:102270008093770126960FB6F894DEBF0FBECDBFD0
:10228000DF91CF911F910F91FF90EF90DF90CF9052
:10229000BF90AF909F900C946E0926960FB6F8945D
:1022A000DEBF0FBECDBFDF91CF911F910F91FF9089
:1022B000EF90DF90CF90BF90AF909F900895CF9315
:1022C000DF93CDB7DEB72B970FB6F894DEBF0FBE06
:1022D000CDBF4F83588769877A878B87DE01119638
:1022E00086E0FD0111928A95E9F785E0FE013796B7
:1022F00001900D928A95E1F749815A816B817C8129
:102300008D819E810E94A8172B960FB6F894DEBF90
:102310000FBECDBFDF91CF910895CF93882309F4ED
:10232000C2C0C82F823859F40E94711081FDBBC011
:1023300089E30E94821A0E944F1B89E30CC08338F4
:1023400079F40E94711080FDAEC083E50E94821A6C
:102350000E944F1B83E50E94C41ACF910C944F1B1F
:10236000843859F40E94711082FD9DC087E40E9458
:10237000821A0E944F1B87E4EECF8CEF8C0F813ABC
:1023800048F48C2F0E94B62081118DC08C2F0E94A2
:10239000821AE3CF80E28C0F883048F4C77081E066
:1023A00001C0880FCA95EAF70E94081BD6CF8BE5BB
:1023B0008C0F833078F4C53A29F0C63A31F083E8BF
:1023C00090E005C081E890E002C082E890E0CF9103
:1023D0000C94931088E58C0F833108F064C0C83AE0
:1023E00039F1C93A41F1CA3A49F1CB3A51F1CC3A03
:1023F00059F1CD3A61F1C03B69F1CE3A71F1CF3A72
:1024000079F1C13B81F1C23B89F1C33B91F1C43BFE
:1024100099F1C53BA1F1C63BA9F1C73BB1F1C83B5E
:10242000B9F1C93BC1F1CA3BC9F180E090E038C0C5
:1024300082EE90E035C089EE90E032C08AEE90E006
:102440002FC085EB90E02CC086EB90E029C087EB95
:1024500090E026C08CEC90E023C08DEC90E020C092
:1024600083E891E01DC08AE891E01AC082E991E01A
:1024700017C084E991E014C081E292E011C083E2C8
:1024800092E00EC084E292E00BC085E292E008C0C8
:1024900086E292E005C087E292E002C08AE292E022
:1024A000CF910C94A910CF910895882309F44BC0C3
:1024B000823859F40E94711081FF45C089E30E945F
:1024C000821A0E944F1B89E30CC0833871F40E946A
:1024D000711080FF38C083E50E94821A0E944F1B52
:1024E00083E50E94C41A0C944F1B843859F40E944F
:1024F000711082FF28C087E40E94821A0E944F1B3D
:1025000087E4EFCF9CEF980F913A58F390E2980F41
:10251000983050F4877091E001C0990F8A95EAF7DE
:10252000892F0E940E1BDFCF9BE5980F933020F47C
:1025300080E090E00C949310885A833120F480E07E
:1025400090E00C94A9100895882321F00E94081BA4
:102550000C944F1B0895882321F00E940E1B0C94AD
:102560004F1B08957F928F929F92AF92BF92CF920E
:10257000DF92EF92FF920F931F93CF93DF931F92FF
:10258000CDB7DEB77C01C62E772EFC010581029502
:102590000F70128111110E94251B0E947B1A882343
:1025A00079F0112369F080E28C0D883048F082E0E8
:1025B0000E94641A0E947B1A91E0D82ED92601C08D
:1025C000D12CE72DE295EF70F0E0E05AFF4F0C942C
:1025D000EA22872D807F072D0F70882311F0029546
:1025E000007F112389F0002309F490C180E28C0D53
:1025F000883020F4802F0E94081B03C0802F0E9487
:10260000181B0E944F1B82C18C2D0E945512002363
:1026100009F495C180E28C0D883020F4802F0E944F
:102620000E1B03C0802F0E941E1B0E944F1B87C1E0
:10263000972D907F872D8F70903211F08295807F3B
:10264000CC2021F0F1E0CF16B1F01EC0112349F0EB
:10265000002309F414C1013009F011C10E94381B94
:102660006EC1002319F0013009F469C189830E9409
:102670003B1B89810AC1112321F0023008F05FC1A0
:10268000FEC001115CC101C1112321F0002309F436
:10269000F6C03CC1002309F4F8C03EC1872D8695E1
:1026A0008695837090E0009719F0019761F047C11B
:1026B000112321F08C2D972D937002C080E090E0C3
:1026C0000E9493103CC1112321F08C2D972D937003
:1026D00002C080E090E00E94A91031C18C2D11232E
:1026E00019F00E94741D02C00E94DC1D0E94611E30
:1026F00026C1872D837009F052C0111120C18C2D85
:10270000829586958770880F880F9C2D9F70892EE3
:10271000912CA12CB12C082E04C0880C991CAA1C49
:10272000BB1C0A94D2F7C4FE14C00FE010E020E0F6
:1027300030E0B901A80104C0440F551F661F771F80
:102740008A95D2F7CB01BA016095709580959095E6
:1027500003C060E070E0CB01272D269526952370FD
:1027600030E02230310569F02330310589F06829E5
:1027700079298A299B292130310571F00E94F018AE
:10278000DEC0682979298A299B290E940C19D7C0A3
:102790000E94F018C501B4010E94D418D0C01123C2
:1027A00019F0872D817001C08695882309F4C7C070
:1027B0008C2D829586958770880F880F9C2D9F7031
:1027C000892E912CA12CB12C082E04C0880C991CA8
:1027D000AA1CBB1C0A94D2F7C4FE14C00FE010E080
:1027E00020E030E0B901A80104C0440F551F661F66
:1027F000771F8A95D2F7CB01BA01609570958095C5
:10280000909503C060E070E0CB01272D26952695BA
:102810002370422F50E04230510569F0433051059A
:1028200089F0682979298A299B294130510571F05D
:102830000E94CA1984C0682979298A299B290E9483
:10284000E6197DC00E94CA19C501B4010E94AE19E3
:1028500076C08C2D90E0FC01E05EF109E531F105D8
:1028600008F050C0E059FF4F0C94EA220C2D0F7075
:10287000872D8F71112331F00E944719802F0E94FC
:10288000A4125DC00E946819802F0E94AB1257C02D
:10289000112339F0011153C0872D8F710E948D19BA
:1028A0004EC0023008F04BC0F7CF112339F0872D0E
:1028B0008F710E94471943C01123C9F3872D8F716F
:1028C0000E9468193CC0112329F0872D8F710E9446
:1028D000321935C00E94281932C0112351F0172D2A
:1028E0001F71812F0E94471963E0812F0E945B1A9C
:1028F00026C081E00E94641A023008F182E00E9442
:10290000641A1DC0112331F0002389F28C2D0E941E
:102910008D1115C0002391F28C2D0E9455120FC00D
:10292000472D4F706C2DC7010E942C050E944C183A
:1029300006C0472D4F706C2DC7010E94DD08DD20B9
:10294000F9F00E94571A80FD1BC0F70112820E9405
:10295000511A0E944719C7010E94CF140E94511AB0
:102960000F90DF91CF911F910F91FF90EF90DF902B
:10297000CF90BF90AF909F908F907F900C946819EC
:102980000F90DF91CF911F910F91FF90EF90DF900B
:10299000CF90BF90AF909F908F907F9008950F93AE
:1029A0001F93CF93DF93EC01888199812B813C8128
:1029B000232BB9F09F3F11F48F3F99F0CE010E9475
:1029C0006E05882371F0688179818A810E944D1A91
:1029D0008C010E94021A0E94C918B801CE010E94FF
:1029E000B212DF91CF911F910F9108950E94251B84
:1029F0000E94351B0E94FA1A0E944F1B0E94121F50
:102A00000E94611E80E090E00E94931080E090E0C0
:102A10000C94A9100E94151B0C94F6140E94421AE3
:102A2000292F22952F7030E02C3031054CF42A30BC
:102A300031056CF42250310922303105A8F407C069
:102A40002C30310569F02F30310551F00DC0803F39
:102A500069F018F4803E40F409C0843F29F406C0B0
:102A600093FB882780F9089580E0089581E0089518
:102A7000CF93DF9300D000D01F92CDB7DEB70F9079
:102A80000F900F900F900F90DF91CF910895CF93FB
:102A9000DF9300D000D000D0CDB7DEB726960FB6BA
:102AA000F894DEBF0FBECDBFDF91CF9108951F9385
:102AB000CF93DF93C091860116E080918701C817FC
:102AC00099F0D0E01C9FF0011D9FF00D1124E857F4
:102AD000FE4F4081518162817381848195810E9482
:102AE00047152196C770E9CFDF91CF911F910895C7
:102AF0004091B8015091B9016091BA017091BB0148
:102B00008091BC019091BD010C9447158091BD014D
:102B100082958F7009F054C08091BA01882309F41E
:102B20004FC080918601A09187016091B80170919A
:102B3000B9014091BB015091BC01B6E08A1709F47C
:102B40003FC090E041155105C1F17F3F11F46F3F47
:102B5000A1F1B89FF001B99FF00D1124E857FE4F85
:102B6000218172132AC02081621327C02281211182
:102B700024C0238134812417350710F421503109F2
:102B8000241B350B283C3105C0F42091BD012F706A
:102B900020612093BD0126E0289FF001299FF00DC0
:102BA0001124E357FE4F80818F708061808388EB12
:102BB00091E00E94CF140C94571501968770BECFF8
:102BC0000895CF92DF92EF92FF920F931F93CF93CE
:102BD000DF93CDB7DEB762970FB6F894DEBF0FBEB6
:102BE000CDBF8C0185E0F801DE011D9601900D92AC
:102BF0008A95E1F7D8014C9111965C911197129644
:102C00006C9112971396CD90DC9014973091B80187
:102C10007091B9018091BB019091BC01009709F4BA
:102C20006BC17F3F19F43F3F09F466C1E090BA01E0
:102C3000EE2009F4C0C02091BD01C816D90628F0C5
:102C4000F601E81BF90BCF0104C0809590958C0D1F
:102C50009D1DFF24F394883C910578F0F12C207F92
:102C600009F0C6C07C2DD98AC88A89890E94381586
:102C700088EB91E00E94CF14B1C0822F807F09F0D1
:102C800046C0751314C0341312C0611110C02F70E8
:102C900020612093BD010E94781588EB91E00E948D
:102CA000CF148091BD01D80115968C932EC0CD28EC
:102CB00019F15F3F11F44F3FF9F0F62E61111CC07E
:102CC000809186012091870136E0821709F45AC06D
:102CD00090E0389FF001399FF00D1124E857FE4F26
:102CE0007181571306C07081471303C0728171113F
:102CF00003C001968770E9CFF62E662309F418C148
:102D00008091BD0181608093BD01F12C11C17513CB
:102D100008C0341306C0611104C08091BD01D80100
:102D2000C3C04D875E878D859E856A8B0E940E1578
:102D30006A898823E1F16623D1F12091BD01822FB8
:102D400082958F7090E0029774F08091B801909115
:102D5000B90198878F831986DB86CA862C87CE01B6
:102D600007960E94CF1486E0F801A8EBB1E001902D
:102D70000D928A95E1F70E9486150E947815FF242E
:102D8000F394D6C04D875E878D859E850E94421A3A
:102D9000292F22952F7030E0223031050CF0BCC075
:102DA0009F7009F0B6C0805E883008F4C1C0C801C9
:102DB0000E94CF14E4CFC816D90608F453C0F60118
:102DC000E81BF90BCF01883C910508F450C0F12CA9
:102DD0007C2DD98AC88A89890E943815E8EBF1E0F0
:102DE00086E0DF011D928A95E9F70E947815A0C060
:102DF000751314C0341312C0611110C08091BD014D
:102E0000F8018583C8010E94CF1486E0E8EBF1E069
:102E1000DF011D928A95E9F7FE2C8AC04D875E87F7
:102E20008D859E856A8B0E940E156A89882309F418
:102E3000BECF662309F4BBCF2091BD01822F8295BE
:102E40008F7090E002970CF48ECF8091B801909132
:102E5000B9019A8389831B82DD82CC822E83CE01C5
:102E600001967FCF809590958C0D9D1DACCFF62E51
:102E7000662309F49CCF75132EC034132CC0209107
:102E8000BD0120FD1FC0822F82958F70D9F0D8011F
:102E900015962C9315978F3049F08F5F982F929548
:102EA000907F822F8F70892B15968C93C8010E947A
:102EB000CF1486E0F801A8EBB1E001900D928A955D
:102EC000E1F793CF86E0F801A8EBB1E001900D9215
:102ED0008A95E1F72DC04D875E878D859E850E947E
:102EE0000E15811140CF8091BD0181608093BD019D
:102EF000C8010E94CF141CC0662309F458CF4D8727
:102F00005E878D859E850E940E15882309F44FCF1C
:102F10002ACF811148CF0CC0243031050CF047CFA7
:102F20009F7009F440CFF8019581907F09F03BCF65
:102F30008F2D62960FB6F894DEBF0FBECDBFDF9126
:102F4000CF911F910F91FF90EF90DF90CF90089558
:102F50001F93CF93DF93CDB7DEB72C970FB6F894BE
:102F6000DEBF0FBECDBF4F83588769877A878B87B7
:102F70009C87CE0107960E94E115882369F08F8116
:102F800098852A853B85232BF1F19F3F09F063C08B
:102F90008F3F09F060C037C086E0FE013796DE0142
:102FA000119601900D928A95E1F76F817885EA85F7
:102FB000FB85309741F17F3F11F46F3F21F1209164
:102FC000870130E0C90101968770992740918601F9
:102FD00050E08417950709F447C069837A83FD831D
:102FE000EC8396E0929FD001939FB00D1124A857D7
:102FF000BE4FFE01319601900D929A95E1F78093B4
:1030000087010E94571516E08091860190918701F3
:103010008917C1F1189FC001112488579E4F0E9443
:10302000E115882379F1E09186011E9FF0011124BA
:10303000E857FE4F4081518162817381848195817F
:103040000E9447158091860190E00196877099272C
:1030500080938601D9CF4F81588569857A858B8584
:103060009C850E944715CFCF0E940A1510928701B8
:1030700010928601E8EBF1E086E0DF011D928A956F
:10308000E9F7C1CF2C960FB6F894DEBF0FBECDBFC7
:10309000DF91CF911F910895EF92FF920F931F93AD
:1030A000CF93DF938C01009709F46CC0F12CEE24D0
:1030B000E394E8012196F8018491843740F4843048
:1030C00008F051C0813081F0823019F15BC0853742
:1030D00009F444C0A8F19CE7980F903708F052C05B
:1030E0008F770E94551241C00E5F1F4FFE01C491A1
:1030F00080E28C0F883048F4C7708E2D01C0880F95
:10310000CA95EAF70E94281B14C08C2F0E948D11CB
:103110002DC00E5F1F4FFE01C49180E28C0F8830DE
:1031200058F4C7708E2D01C0880FCA95EAF70E9427
:103130002E1B0E944F1B1AC08C2F0E94551216C0C6
:103140000E5F1F4FFE01C491CC2381F08FE99FE0F9
:103150000197F1F700C00000C150F6CF0E5F1F4F7E
:10316000FE01F49003C00E948D118E018F2D8823E3
:1031700009F49FCFEFE9FFE03197F1F700C00000BD
:103180008150F5CFDF91CF911F910F91FF90EF907C
:10319000089508956093C2017093C3018093C401A0
:1031A0009093C5010C94F6140F931F930091C201E4
:1031B0001091C3012091C4013091C501DC01CB0104
:1031C000802B912BA22BB32B8093C2019093C30130
:1031D000A093C401B093C5011F910F910C94F614F4
:1031E0000F931F930091C2011091C3012091C4015C
:1031F0003091C501DC01CB0180239123A223B323AD
:103200008093C2019093C301A093C401B093C50100
:103210001F910F910C94F6140F931F930091C2010C
:103220001091C3012091C4013091C501DC01CB0193
:1032300080279127A227B3278093C2019093C301CF
:10324000A093C401B093C5011F910F910C94F61483
:103250001092BE011092BF011092C0011092C101E4
:103260000C94F61441E050E060E070E004C0440FBC
:10327000551F661F771F8A95D2F74093BE01509362
:10328000BF016093C0017093C1010C94F61441E03A
:1032900050E060E070E004C0440F551F661F771FC8
:1032A0008A95D2F78091BE019091BF01A091C00193
:1032B000B091C101482B592B6A2B7B2B4093BE0147
:1032C0005093BF016093C0017093C1010C94F61438
:1032D00041E050E060E070E004C0440F551F661FFD
:1032E000771F8A95D2F7409550956095709580919B
:1032F000BE019091BF01A091C001B091C1014823CE
:1033000059236A237B234093BE015093BF016093EE
:10331000C0017093C1010C94F61441E050E060E0EC
:1033200070E004C0440F551F661F771F8A95D2F7BF
:103330008091BE019091BF01A091C001B091C101E7
:10334000482759276A277B274093BE015093BF0126
:103350006093C0017093C1010C94F6140F931F93F6
:103360000091BE011091BF012091C0013091C101B7
:10337000DC01CB01802B912BA22BB32B8093BE01C0
:103380009093BF01A093C001B093C1011F910F9111
:103390000C94F6140F931F930091BE011091BF017E
:1033A0002091C0013091C101DC01CB018023912328
:1033B000A223B3238093BE019093BF01A093C001C9
:1033C000B093C1011F910F910C94F6140F931F93AA
:1033D0000091BE011091BF012091C0013091C10147
:1033E000DC01CB0180279127A227B3278093BE0160
:1033F0009093BF01A093C001B093C1011F910F91A1
:103400000C94F6140895CF92DF92EF92FF920F93EF
:103410001F93CF93DF938C01C090C201D090C30162
:10342000E090C401F090C5018091BE019091BF0170
:10343000A091C001B091C101C82AD92AEA2AFB2A69
:10344000CFE1D0E0D701C6010C2E04C0B695A795F8
:10345000979587950A94D2F780FF06C0B8018C2F04
:103460000E945C07019721F4219760F780E001C07A
:103470008C2FDF91CF911F910F91FF90EF90DF90F4
:10348000CF900895CF93DF93EC010E94031ABE0101
:103490000E945C07DF91CF910895CB010E94421AF0
:1034A00008958091C60185958595859508958091AB
:1034B000C6018770089598E0899F90011124262BFA
:1034C0002093C6010C9447192091C6018095822350
:1034D0008093C601982F977069F430E0482F5527E4
:1034E00047FD50952417350729F0859585958595D5
:1034F0000C94681908959091C601977081E009F4C1
:1035000080E0089590910C01992321F090910D0194
:10351000911109C020910E0130910F01F9013296ED
:103520009FEF40E01FC0982F9695969596959F30F7
:1035300050F5E0910E01F0910F01E90FF11D877038
:1035400021E030E0A90102C0440F551F8A95E2F73F
:10355000CA019181892B818308959F3F39F04F5F84
:103560004E3041F051915813F8CF0DC05111F7CFA3
:10357000942FF5CF9F3F39F0F901E90FF11D97FD29
:10358000FA9582830895089590910C01992321F072
:1035900090910D01911109C020910E0130910F0100
:1035A000F9013296205F3F4F1FC0982F9695969550
:1035B00096959F30F0F4E0910E01F0910F01E90F24
:1035C000F11D877021E030E0A90102C0440F551FB2
:1035D0008A95E2F7CA0180959181892381830895B4
:1035E0003196E217F30729F090819813F9CF1082F2
:1035F000F7CF089581E090E0E0910E01F0910F0186
:10360000E80FF91F1082019680319105A9F70895FE
:103610009091DA01892B8093DA0108958095909139
:10362000DA0189238093DA0108951092DA0108956E
:103630009091D901892B8093D9010895809590911B
:10364000D90189238093D90108951092D901089551
:103650009091D801892B8093D801089580959091FD
:10366000D80189238093D80108951092D801089534
:103670008093C70108951092C701089580910E01AB
:1036800090910F01FC0131969C01205F3F4F80E03B
:10369000919191118F5FE217F307D1F70895E091AF
:1036A0000E01F0910F018091DA018083E0910E010B
:1036B000F0910F0190818091D901892B8083E09155
:1036C0000E01F0910F0190818091D801892B8083A8
:1036D0008091C701882361F0E0910E01F0910F0104
:1036E0009081892B80830E943E1B81111092C7011B
:1036F00080910E0190910F010C947D1020E00097B5
:1037000039F0AC0141505109842395232F5FF7CF45
:10371000822F0895CF92DF92EF92FF926C01EE24F8
:10372000FF24C114D104E104F10421F0C701B60162
:1037300020E101C020E0C72ED82EE92EFF24C114BD
:10374000D104E104F10419F0285FC701B6016B014F
:103750007C0154E0F694E794D794C7945A95D1F736
:10376000C114D104E104F10419F02C5FC701B601C2
:103770006B017C0142E0F694E794D794C7944A9594
:10378000D1F7C114D104E104F10419F02E5FC7018F
:10379000B601DC01CB01B695A79597958795892B46
:1037A0008A2B8B2B09F02F5F822FFF90EF90DF90F9
:1037B000CF9008958091F401843021F11092DC01C2
:1037C00020E488E190E00FB6F894A895809360001B
:1037D0000FBE2093600080E00E946E0983B7817F56
:1037E000846083BF83B7816083BF7894889583B7F3
:1037F0008E7F83BF88E10FB6F894809360001092AB
:1038000060000FBE089508950E944F030E94620356
:103810000E94031C0E94570491E0811101C090E0B6
:10382000892F08950E940A150E9471100C946E0948
:1038300082E084BD93E095BD9AEF97BD80936E00C2
:1038400008952FB7F8948091DD019091DE01A09149
:10385000DF01B091E0012FBF0895CF92DF92EF9288
:10386000FF920F931F932FB7F8944091DD01509171
:10387000DE016091DF017091E0012FBF6A017B01E1
:10388000EE24FF248C0120E030E0C016D106E206D1
:10389000F30610F4415051099A01281B390BC90154
:1038A0001F910F91FF90EF90DF90CF9008951F929E
:1038B0000F920FB60F9211248F939F93AF93BF93E4
:1038C0008091DD019091DE01A091DF01B091E001D6
:1038D0000196A11DB11D8093DD019093DE01A0939F
:1038E000DF01B093E001BF91AF919F918F910F9055
:1038F0000FBE0F901F9018950E946E0DF8942FEF39
:1039000087EA91E6215080409040E1F700C0000036
:1039100087E090EBDC018093FD019093FE01A09382
:10392000FF01B09300029CE088E10FB6F894A895DF
:10393000809360000FBE90936000FFCF0E94D61C62
:10394000811102C00E94BC1C0E94E11C8093DB011B
:103950000E94E91C90E09093EF018093EE0187FBB9
:10396000882780F980930D010E94E51C682F70E084
:1039700080E090E00C94CA186DEE7EEF80E090E05D
:103980000E94242360E082E090E00E94122360E025
:1039900083E090E00E94122360E084E090E00E94C7
:1039A000122360E085E090E00C94122380E090E028
:1039B0000E940C2321E08D3E9E4F09F020E0822FD3
:1039C000089582E090E00C94042383E090E00C944E
:1039D000042384E090E00C940423682F84E090E0BA
:1039E0000C9412238091E30180FF0BC060911301BE
:1039F00085E0689FB0011124759567957595679569
:103A00002BC081FF09C06091130185E0689FB00160
:103A100011247595679520C082FF07C0609113013E
:103A200085E0689FB001112417C09091E4019923AB
:103A3000D1F060911201961788F72091130185E06B
:103A4000289F90011124929FA001939F500D112453
:103A500070E0CA010E94D6226038710540F46115F9
:103A6000710539F002C065E070E0862F08958FE798
:103A7000089581E008958091E30180FF08C060917E
:103A8000110170E0759567957595679521C081FF67
:103A900006C06091110170E07595679519C082FFAD
:103AA00004C06091110170E010C09091E40199236D
:103AB000C1F0609110019617A0F780911101899FC4
:103AC000C001112470E00E94D6226038710528F4EC
:103AD0006115710521F0862F08958FE7089581E023
:103AE000089561E070E0F4CF803F21F40E94F21C61
:103AF000819504C0813F29F40E94F21C8093E70164
:103B00000895823F21F40E94F21C819504C0833FF6
:103B100029F40E94F21C8093E6010895893F19F46C
:103B20000E943B1D05C08A3F31F40E943B1D8195D8
:103B30008093E80108958B3F21F40E943B1D8195FD
:103B400004C08C3F29F40E943B1D8093E901089535
:103B5000843F21F48091E501816017C0853F21F405
:103B60008091E501826011C0863F21F48091E501DA
:103B700084600BC0873F21F48091E501886005C017
:103B8000883F31F48091E50180618093E5010895DB
:103B90008D3F21F48091E30181600BC08E3F21F4C1
:103BA0008091E301826005C08F3F29F48091E30199
:103BB00084608093E3010895803F39F48091E701A8
:103BC00087FF6CC01092E70169C0813F29F48091A2
:103BD000E7011816BCF362C09091E601823F29F418
:103BE00097FF5CC01092E60159C0833F19F4191683
:103BF000CCF354C0893F41F48091E80118160CF0D1
:103C00004DC01092E8014AC08A3F29F48091E80132
:103C100087FF44C0F6CF8B3F39F48091E90187FFDD
:103C20003DC01092E9013AC08C3F29F48091E9012E
:103C30001816BCF333C0843F21F48091E5018E7FD8
:103C400017C0853F21F48091E5018D7F11C0863F2B
:103C500021F48091E5018B7F0BC0873F21F4809197
:103C6000E501877F05C0883F31F48091E5018F7EB3
:103C70008093E50113C08D3F21F48091E3018E7F95
:103C80000BC08E3F21F48091E3018D7F05C08F3FF3
:103C900029F48091E3018B7F8093E3018091E60119
:103CA00081110EC08091E70181110AC08091E80165
:103CB000811106C08091E901811102C01092E401D6
:103CC000089585EE91E00E9488100E94211C909337
:103CD000E2018093E10108951F93CF93DF938091D8
:103CE000E1019091E2010E942D1CAC019091E40150
:103CF000992321F02091140130E006C02091150194
:103D00008AE0289F900111244217530708F486C0C7
:103D10008091E601C091E701D091E8011091E9019D
:103D2000811107C0C11176C0D11174C0111172C0C8
:103D300075C09F3F19F09F5F9093E401181624F41B
:103D40000E94F21C8093E6018091E60187FF05C086
:103D50000E94F21C81958093E6011C1624F40E94B7
:103D6000F21C8093E7018091E70187FF05C00E9464
:103D7000F21C81958093E7016091E601662339F199
:103D8000C091E701CC2319F1772767FD7095872F44
:103D9000972F0E94E72123E333E343E35FE30E948D
:103DA0004B220E94B4216093E6016C2F772767FDB8
:103DB0007095872F972F0E94E72123E333E343E396
:103DC0005FE30E944B220E94B4216093E7011D161D
:103DD00024F40E943B1D8093E8018091E80187FF55
:103DE00005C00E943B1D81958093E801111624F4C3
:103DF0000E943B1D8093E9018091E90187FF05C086
:103E00000E943B1D81958093E901DF91CF911F9125
:103E10000C94611E9F3F09F08ECF96CFDF91CF911A
:103E20001F910895E5EEF1E085E0DF011D928A958E
:103E3000E9F71092E4011092E3010895833081F1D3
:103E400028F4813059F08230D1F00895853009F49A
:103E500049C0B8F1863009F456C008958091150123
:103E6000262F30E0280F311D2F3F310524F4680F35
:103E70006093150108958FEF809315010895809147
:103E80001401262F30E0280F311D2F3F310524F477
:103E9000680F6093140108958FEF809314010895C3
:103EA00080911301262F30E0280F311D2F3F31055F
:103EB00024F4680F6093130108958FEF809313012A
:103EC000089580911201262F30E0280F311D2F3FD9
:103ED000310524F4680F6093120108958FEF8093E9
:103EE0001201089580911101262F30E0280F311D15
:103EF0002F3F310524F4680F6093110108958FEF6F
:103F000080931101089580911001262F30E0280F31
:103F1000311D2F3F310524F4680F6093100108957F
:103F20008FEF809310010895833011F128F48130D0
:103F300049F0823091F00895853081F120F186308A
:103F4000C1F1089580911501681720F4861B8093B4
:103F500015010895109215010895809114016817B4
:103F600020F4861B80931401089510921401089583
:103F700080911301681720F4861B80931301089524
:103F800010921301089580911201681720F4861B86
:103F900080931201089510921201089580911101E9
:103FA000681720F4861B8093110108951092110167
:103FB000089580911001681720F4861B80931001EA
:103FC00008951092100108950F931F938D3109F4F5
:103FD00071C008F045C0803109F485C008F587300C
:103FE00009F46FC068F4863009F0ADC08091DB0140
:103FF000817F8E7F8093DB0181E08093EB01A4C001
:104000008B3009F49EC08E3009F09DC08091DB0199
:1040100082FB222720F991E0922790FB82F96CC065
:10402000863109F48EC060F4813109F08CC00E94A1
:104030000A1590910D0181E0892780930D0181C0BF
:10404000893109F47EC08B3109F07DC08091DB019C
:1040500081FB222720F991E0922790FB81F94CC047
:10406000853309F466C048F4873209F462C008F465
:104070004FC0893209F45DC066C0833438F48A3396
:1040800008F044C0883309F45CC05DC0833409F48F
:1040900050C0883409F057C00E940A150FEF13ED85
:1040A00020E3015010402040E1F700C000000E94D2
:1040B0007C1C47C00E946E210E9471100E946E09F4
:1040C00040C09091DB01892F8095817080FB90F931
:1040D00029F0966098609093DB0136C0997F977FB6
:1040E0009093DB012EC08091DB0183FB222720F916
:1040F00091E0922790FB83F98093DB01992309F1EA
:104100008091DB0181608093DB011BC0895301C07A
:104110008D5141E050E060E070E08A019B0104C0F5
:10412000000F111F221F331F8A95D2F7C901B80152
:1041300004C061E070E080E090E00E94CA180E9434
:104140000A1581E001C080E01F910F91089580E081
:10415000089580E008958E518A3030F4E82FF0E021
:10416000E65DFE4F8081089580E00895CF93C82FCB
:104170008091EB01813079F018F08230E9F186C04E
:10418000E0910E01F0910F018081813169F082325E
:1041900009F07EC009C0E0910E01F0910F0180810D
:1041A000813111F0823261F48C2F0E94A72081119D
:1041B00004C08C2F0E94E41F1DC081E090E01AC053
:1041C0008C2F0E94A920811114C0C43179F048F4C9
:1041D000CB3079F0C03109F05FC082E08093EB0111
:1041E00008C0C93219F0C83321F056C01092EB0153
:1041F00053C081E0817052C0C93281F110F5C431E1
:1042000069F1A8F4C73009F045C08AE08093150130
:1042100094E19093140193E0909313018093120121
:1042200088E08093110188E28093100133C082EE10
:104230008C0F863078F58C2F0E94AB208093EA019A
:1042400029C0CE34E9F020F4CB3421F56AE013C064
:10425000C13579F0C235F1F461E00DC08091EA0119
:10426000882319F01092EA0115C081E08093EB01D8
:1042700015C061E006C08091EA010E941E1F0AC0BD
:104280006AE08091EA010E94941F04C01092EB0141
:1042900080E004C081E002C080E0ACCFCF910895FF
:1042A000E1E8F0E0808188608083808181608083A4
:1042B0008FB7F89493E09093890090ED90938800E5
:1042C0008FBF0895EFE6F0E08081826080830895DB
:1042D000EFE6F0E080818D7F80830895EFE6F0E0E7
:1042E000908182E08927808308951F920F920FB6F4
:1042F0000F9211242F933F934F935F936F937F936C
:104300008F939F93AF93BF93EF93FF938091EC01B3
:104310009091ED0101969093ED018093EC01811154
:1043200003C082E00E946E09E091ED01E695E695FA
:10433000F0E0EB54FB4FE4918091EC018E1303C04D
:1043400080E00E946E09FF91EF91BF91AF919F9124
:104350008F917F916F915F914F913F912F910F902E
:104360000FBE0F901F90189504D06894B1118DC0A6
:10437000089570D088F09F5790F0B92F9927B751C2
:10438000A0F0D1F0660F771F881F991F1AF0BA9519
:10439000C9F712C0B13081F077D0B1E0089574C090
:1043A000672F782F8827B85F39F0B93FCCF386950F
:1043B00077956795B395D9F73EF49095809570956C
:1043C00061957F4F8F4F9F4F0895E89409C097FBE9
:1043D0003EF490958095709561957F4F8F4F9F4FDC
:1043E0009923A9F0F92F96E9BB279395F695879520
:1043F00077956795B795F111F8CFFAF4BB0F11F4E3
:1044000060FF1BC06F5F7F4F8F4F9F4F16C0882389
:1044100011F096E911C0772321F09EE8872F762FBF
:1044200005C0662371F096E8862F70E060E02AF000
:104430009A95660F771F881FDAF7880F96958795EC
:1044400097F9089557FD9058440F551F59F05F3F55
:1044500071F04795880F97FB991F61F09F3F79F0A6
:1044600087950895121613061406551FF2CF469528
:10447000F1DF08C0161617061806991FF1CF8695AA
:104480007105610508940895E894BB27662777278E
:10449000CB0197F908950BD078C069D028F06ED081
:1044A00018F0952309F05AC05FC01124EECFCADF7F
:1044B000A0F3959FD1F3950F50E0551F629FF00137
:1044C000729FBB27F00DB11D639FAA27F00DB11D90
:1044D000AA1F649F6627B00DA11D661F829F222719
:1044E000B00DA11D621F739FB00DA11D621F839FA0
:1044F000A00D611D221F749F3327A00D611D231F76
:10450000849F600D211D822F762F6A2F11249F57C3
:1045100050408AF0E1F088234AF0EE0FFF1FBB1FE6
:10452000661F771F881F91505040A9F79E3F510585
:1045300070F014C0AACF5F3FECF3983EDCF3869591
:1045400077956795B795F795E7959F5FC1F7FE2B30
:10455000880F911D9695879597F9089597F99F670C
:1045600080E870E060E008959FEF80EC08950024FB
:104570000A941616170618060906089500240A94C8
:1045800012161306140605060895092E0394000C4E
:1045900011F4882352F0BB0F40F4BF2B11F460FFDD
:1045A00004C06F5F7F4F8F4F9F4F089597FB072E7B
:1045B00016F4009407D077FD09D00E94F02207FC82
:1045C00005D03EF4909581959F4F08957095619523
:1045D0007F4F0895EE0FFF1F0590F491E02D099491
:1045E000AA1BBB1B51E107C0AA1FBB1FA617B70719
:1045F00010F0A61BB70B881F991F5A95A9F7809535
:104600009095BC01CD010895F999FECF92BD81BD71
:10461000F89A992780B50895A8E1B0E042E050E00B
:104620000C942C23262FF999FECF92BD81BDF89AC8
:10463000019700B4021639F01FBA20BD0FB6F894E6
:10464000FA9AF99A0FBE08950196272F0E94132314
:104650000C941223DC01CB01FC01F999FECF06C0BA
:10466000F2BDE1BDF89A319600B40D924150504030
:08467000B8F70895F894FFCF9C
:1046780002207009FE09DB09A70973090101C801B5
:1046880028080A03140A404D363975042804F20331
:10469800B9034C0365037E0397030102030405066F
:0446A80007080900F6
:00000001FF
